:020000040000FA
:040000008FEF00F08E
:020008009ED088
:08001800ECD00E6E960E066E90
:10002000980E076E55D8D8B4CA90D8A4CA80FC0FD1
:10003000D8A0CA92D8B0CA82800E066E960E076EFD
:10004000980E0A6E0B6ACAB025D8CAB223D842D815
:100050000604CB6E06C008F007C009F000500C6E15
:100060000D6E003C0D6A4BD80B500E2E0AD0BE6EA2
:100070000C0EBD6E0ABEBD8A0ABCBD889394CA84AC
:100080001200BB6E0C0EBA6E0ABEBA8A0ABCBA88DF
:100090009492F5D700D8D8900A320732063212006F
:1000A000096A086EFF0E0826092200D0D8A01200A7
:1000B000030E076EE70E02D8F5D7076AFE0F066E2D
:1000C000E86A075AD8A012000000060600D0F8D748
:1000D0000B6A0A6A100EF36E07340A360B360850A4
:1000E0000A5C09500B5805E308500A5E09500B5A88
:1000F000D88006360736F32EEFD706501200085088
:100100000C02F3CF0AF0F4CF0BF009500C02F350BD
:100110000B2608500D02F3500B260A501200F86A05
:100120004F0EAF6E240EAC6E900EAB6E0001C69AF1
:10013000430E926EE00E936EC00E946E070EB46E78
:100140000F0EC16E9DD09EAA1BD0060EAB1412E1FD
:10015000E1CF35F0E2CF36F0372A1EEE80F037508F
:10016000E126000EE222AECFE7FF35C0E1FF36C048
:10017000E2FF1100AE50AE50AB98AB8811000AD030
:10018000F2A408D0F294114A122A817A106AD6CFCA
:100190000FF0110011003750385C14E0382AE9CF15
:1001A00006F0EACF07F00EEE80F03850E926000E98
:1001B000EA22EF50066E06C0E9FF07C0EAFFD880CA
:1001C000120004D0E868066ED8A012001200376A48
:1001D000386A9D8A9F8AF28EF28C12009D9A0EEEEA
:1001E00080F0000EEE6AE82EFDD7376A386A9D8AE5
:1001F0001200F29ED8CF5AFEE8CF5BFEE0CF5CFE45
:10020000E9CF5DFEEACF5EFEE1CF5FFEE2CF60FEAA
:10021000D9CF61FEDACF62FEF6CF63FEF7CF64FE80
:10022000F5CF65FEF3CF66FEF4CF67FEA6CF68FE7E
:10023000F28E0001A192F29E5ACED8FF5BCEE8FF6B
:100240005CCEE0FF5DCEE9FF5ECEEAFF5FCEE1FF70
:1002500060CEE2FF61CED9FF62CEDAFF63CEF6FF59
:1002600064CEF7FF65CEF5FF66CEF3FF67CEF4FFF1
:1002700068CEA6FFF28E10009EA8FED7AD6E1200CB
:100280009298899893948A94949A8B9A94988B983C
:1002900094968B9694948B9494928B9294908B904A
:1002A000929A899A2A6A2B6A2C6A2D6A2E6A2F6A78
:1002B000306A316A326A336A929489949296899646
:1002C000939A8A9A006A280E086E260E096E020E0C
:1002D000A4DE006A280E086E260E096E010E9DDE51
:1002E000256AC4EC06F0C1EC08F0939A8A8A320EB3
:1002F000D7DE939A8A9A236A6ADF70DFCD6AF29416
:10030000F28A870ED56EB16AA192A082D08EA29297
:10031000B00EB16E40DF136EBE0E135C07E3FE0E2F
:10032000135C02E302D202D0156AFFD113AE21D0D2
:10033000156A8D0E135C05E113C015F01668176879
:1003400017D09D0E135C05E113C015F018681968ED
:100350000FD0AD0E135C05E113C015F01A681B68D1
:1003600007D0BD0E135C04E113C015F01C681D68B6
:10037000DCD1155202E1D9D1D8D18D0E155CD8A4AB
:1003800040D0162803E113C016F039D03D0E165C9C
:1003900004E123908B9A299031D03E0E165C04E143
:1003A00023928B9829922AD03F0E165C04E1239465
:1003B0008B96299423D0400E165C04E123968B90F3
:1003C00029961CD0420E165C04E12398899A29983C
:1003D00015D07E0E165C08E1006A280E086E260E07
:1003E000096E010E1ADE0AD07F0E165C07E1006A64
:1003F000280E086E260E096E020E0FDE166895D1C5
:1004000094D19D0E155CD8A475D1182803E113C0B2
:1004100018F06ED113C019F019523CE13D0E185C72
:1004200004E123908B9A299033D03E0E185C04E1AE
:1004300023928B9829922CD03F0E185C04E12394D0
:100440008B96299425D0400E185C04E123968B905E
:1004500029961ED0420E185C04E12398899A2998A7
:1004600017D07E0E185C09E1006A280E086E260E71
:10047000096E010E0DEC00F00BD07F0E185C08E148
:10048000006A280E086E260E096E020E0DEC00F0B2
:1004900018684BD13D0E185C33E12A5202E12B5211
:1004A000D8A429802380D6CF0FF0D7CF10F002EE4A
:1004B0006BF0D8901934E926000EEA22EECF01F055
:1004C000EFCF02F001C039F002C03AF039C001F0BC
:1004D0003AC002F001500F241F6E02501020206E0F
:1004E000000E1120216E000E1220226E21C043F05A
:1004F00022C044F01FC04DF020C04EF08B8AF7D0D0
:100500003E0E185C33E12C5202E12D52D8A4298210
:100510002382D6CF0FF0D7CF10F003EE6BF0D89038
:100520001934E926000EEA22EECF01F0EFCF02F0F7
:1005300001C03BF002C03CF03BC001F03CC002F007
:1005400001500F241F6E02501020206E000E11204B
:10055000216E000E1220226E21C045F022C046F00E
:100560001FC04FF020C050F08B88C1D03F0E185CE8
:1005700033E12E5202E12F52D8A429842384D6CF0E
:100580000FF0D7CF10F004EE6BF0D8901934E926B5
:10059000000EEA22EECF01F0EFCF02F001C03DF0F5
:1005A00002C03EF03DC001F03EC002F001500F24F9
:1005B0001F6E02501020206E000E1120216E000EC2
:1005C0001220226E21C047F022C048F01FC051F017
:1005D00020C052F08B868BD0400E185C33E1305235
:1005E00002E13152D8A429862386D6CF0FF0D7CF87
:1005F00010F005EE6BF0D8901934E926000EEA22CF
:10060000EECF01F0EFCF02F001C03FF002C040F0AA
:100610003FC001F040C002F001500F241F6E025095
:100620001020206E000E1120216E000E1220226E6E
:1006300021C049F022C04AF01FC053F020C054F03E
:100640008B8055D0420E185C33E1325202E13352B6
:10065000D8A429882388D6CF0FF0D7CF10F006EE84
:100660006BF0D8901934E926000EEA22EECF01F0A3
:10067000EFCF02F001C041F002C042F041C001F0F2
:1006800042C002F001500F241F6E02501020206E55
:10069000000E1120216E000E1220226E21C04BF0A0
:1006A00022C04CF01FC055F020C056F0898A1FD0E0
:1006B0007E0E185C0DE1D8901934346E34C000F011
:1006C000280E086E260E096E010E0DEC00F00FD0FC
:1006D0007F0E185C0CE1D8901934346E34C000F0F1
:1006E000280E086E260E096E020E0DEC00F018683A
:1006F0001CD01BD0AD0E155C0BE11A2803E113C012
:100700001AF004D013C01BF0E3EC05F00ED00DD0AE
:10071000BD0E155C0AE11C2803E113C01CF004D0D7
:1007200013C01DF048EC06F000D023A03CD043C01D
:1007300021F044C022F04DC01FF04EC020F0D6CFB3
:100740000FF0D7CF10F01F500F5C205010582150E1
:1007500011582250125812502218D8B0800A22E79D
:100760008B9A239029A01ED02A5202E12B5219E025
:10077000D6CF0FF0D7CF10F02A500F241F6E2B507A
:100780001020206E000E1120216E000E1220226E0D
:1007900021C057F022C058F01FC061F020C062F0A5
:1007A00001D0299035D029A033D057C021F058C0AE
:1007B00022F061C01FF062C020F0D6CF0FF0D7CF7B
:1007C00010F01F500F5C205010582150115822502B
:1007D000125812502218D8B0800A1AE7238039C064
:1007E00001F03AC002F001500F241F6E0250102099
:1007F000206E000E1120216E000E1220226E21C0EC
:1008000043F022C044F01FC04DF020C04EF08B8A50
:1008100023A23CD045C021F046C022F04FC01FF0BB
:1008200050C020F0D6CF0FF0D7CF10F01F500F5C84
:10083000205010582150115822501258125022188E
:10084000D8B0800A22E78B98239229A21ED02C527E
:1008500002E12D5219E0D6CF0FF0D7CF10F02C5077
:100860000F241F6E2D501020206E000E1120216EBF
:10087000000E1220226E21C059F022C05AF01FC073
:1008800063F020C064F001D0299235D029A233D082
:1008900059C021F05AC022F063C01FF064C020F09C
:1008A000D6CF0FF0D7CF10F01F500F5C205010584C
:1008B000215011582250125812502218D8B0800AD4
:1008C0001AE723823BC001F03CC002F001500F2424
:1008D0001F6E02501020206E000E1120216E000E9F
:1008E0001220226E21C045F022C046F01FC04FF0FA
:1008F00020C050F08B8823A43CD047C021F048C0D2
:1009000022F051C01FF052C020F0D6CF0FF0D7CF49
:1009100010F01F500F5C20501058215011582250D9
:10092000125812502218D8B0800A22E78B962394CE
:1009300029A41ED02E5202E12F5219E0D6CF0FF07B
:10094000D7CF10F02E500F241F6E2F501020206E86
:10095000000E1120216E000E1220226E21C05BF0CD
:1009600022C05CF01FC065F020C066F001D0299461
:1009700035D029A433D05BC021F05CC022F065C023
:100980001FF066C020F0D6CF0FF0D7CF10F01F5069
:100990000F5C2050105821501158225012581250FC
:1009A0002218D8B0800A1AE723843DC001F03EC067
:1009B00002F001500F241F6E02501020206E000E16
:1009C0001120216E000E1220226E21C047F022C09D
:1009D00048F01FC051F020C052F08B8623A63CD0B7
:1009E00049C021F04AC022F053C01FF054C020F08B
:1009F000D6CF0FF0D7CF10F01F500F5C20501058FB
:100A0000215011582250125812502218D8B0800A82
:100A100022E78B90239629A61ED0305202E1315254
:100A200019E0D6CF0FF0D7CF10F030500F241F6E43
:100A300031501020206E000E1120216E000E122069
:100A4000226E21C05DF022C05EF01FC067F020C0A2
:100A500068F001D0299635D029A633D05DC021F0A9
:100A60005EC022F067C01FF068C020F0D6CF0FF044
:100A7000D7CF10F01F500F5C205010582150115844
:100A80002250125812502218D8B0800A1AE7238632
:100A90003FC001F040C002F001500F241F6E025011
:100AA0001020206E000E1120216E000E1220226EEA
:100AB00021C049F022C04AF01FC053F020C054F0BA
:100AC0008B8023A83CD04BC021F04CC022F055C0F5
:100AD0001FF056C020F0D6CF0FF0D7CF10F01F5028
:100AE0000F5C2050105821501158225012581250AB
:100AF0002218D8B0800A22E7899A239829A81ED004
:100B0000325202E1335219E0D6CF0FF0D7CF10F0B6
:100B100032500F241F6E33501020206E000E112013
:100B2000216E000E1220226E21C05FF022C060F004
:100B30001FC069F020C06AF001D0299835D029A8DB
:100B400033D05FC021F060C022F069C01FF06AC0DE
:100B500020F0D6CF0FF0D7CF10F01F500F5C2050F1
:100B60001058215011582250125812502218D8B043
:100B7000800A1AE7238841C001F042C002F0015008
:100B80000F241F6E02501020206E000E1120216EC7
:100B9000000E1220226E21C04BF022C04CF01FC06C
:100BA00055F020C056F0898A23502924016E026A2C
:100BB00002360250011005E1010E125C02E3116AD7
:100BC000126A8AEF01F03D0E1A5C11E11B520CE033
:100BD00000EE6BF0D8901B34E926000EEA22EECF2F
:100BE0002AF0EFCF2BF002D02A6A2B6A4FD03E0EAC
:100BF0001A5C11E11B520CE000EE6BF0D8901B3434
:100C0000E926000EEA22EECF2CF0EFCF2DF002D035
:100C10002C6A2D6A3BD03F0E1A5C11E11B520CE08E
:100C200000EE6BF0D8901B34E926000EEA22EECFDE
:100C30002EF0EFCF2FF002D02E6A2F6A27D0400E71
:100C40001A5C11E11B520CE000EE6BF0D8901B34E3
:100C5000E926000EEA22EECF30F0EFCF31F002D0DD
:100C6000306A316A13D0420E1A5C10E11B520CE05C
:100C700000EE6BF0D8901B34E926000EEA22EECF8E
:100C800032F0EFCF33F002D0326A336A1A681200C2
:100C9000420E1C5C09E11D5203E124D8256A03D0F1
:100CA00089881DC025F004D07B0E1C5CD8B402D806
:100CB0001C681200236A296A006A280E086E260E34
:100CC000096E010E0DEC00F0006A280E086E260E6B
:100CD000096E020E0DEC00F08B9A8B988B968B9020
:100CE000899A1200236A296A8998006A280E086E78
:100CF000260E096E010E0DEC00F0006A280E086E3B
:100D0000260E096E020E0DEC00F08B9A8B988B96D6
:100D10008B90899A2A6A2B6A2C6A2D6A2E6A2F6A0E
:100D2000306A316A326A336A1200CBEC00F0136E1B
:100D3000BE0E135C04E3FE0E135C01E2156A13AEF3
:100D400009D0156ABD0E135C04E113C015F01C68D0
:100D50001D6814D0BD0E155C11E11C2803E113C001
:100D60001CF00CD013C025F0420E1C5C07E11C687F
:100D7000255204E089888A848AEF01F0010E125C12
:100D800002E3116A126AD1D7C30E6D6EA20E6E6EA7
:100D9000990E6F6E980E706EC20E716E930E726E1B
:100DA000120E736E8F0E746E880E756E8A0E766ECE
:100DB000230E776E860E786EE10E796E810E7A6E56
:100DC000C30E7B6E7D0E7C6EC50E7D6E790E7E6EC3
:100DD000E80E7F6E750E806F2B0E816F720E826F24
:100DE0008B0E836F6E0E846F0A0E856F6B0E866F8F
:100DF000A40E876F670E886F5B0E896F640E8A6F13
:100E00002C0E8B6F610E8C6F160E8D6F5E0E8E6FBB
:100E10001A0E8F6F5B0E906F360E916F580E926F99
:100E20006A0E936F550E946FB40E956F520E966FB7
:100E3000150E976F500E986F8A0E996F4D0E9A6F20
:100E4000140E9B6F4B0E9C6FB30E9D6F480E9E6FE2
:100E5000640E9F6F460EA06F290EA16F440EA26F05
:100E6000A369410EA46FE70EA56F3F0EA66FE00EBB
:100E7000A76F3D0EA86FEA0EA96F3B0EAA6F030E77
:100E8000AB6F3A0EAC6F2C0EAD6F380EAE6F640EBA
:100E9000AF6F360EB06FAA0EB16F340EB26FFE0E8A
:100EA000B36F320EB46F600EB56F310EB66FCF0EEA
:100EB000B76F2F0EB86F4B0EB96F2E0EBA6FD30EE1
:100EC000BB6F2C0EBC6F670EBD6F2B0EBE6F060E78
:100ED000BF6F2A0EC06FB10EC16F280EC26F660EB3
:100EE000C36F270EC46F260EC56FC66FF10EC76F96
:100EF000240EC86FC50EC96F230ECA6FA20ECB6F2A
:100F0000220ECC6F890ECD6F210ECE6F790ECF6F72
:100F1000200ED06F710ED16F1F0ED26F710ED36F76
:100F20001E0ED46F7A0ED56F1D0ED66F8B0ED76F37
:100F30001C0ED86FA30ED96F1B0EDA6FC30EDB6FBA
:100F40001A0EDC6FE90EDD6F190EDE6F170EDF6F04
:100F5000190EE06F4B0EE16F180EE26F860EE36F15
:100F6000170EE46FC70EE56F160EE66F0E0EE76FF5
:100F7000160EE86F5B0EE96F150EEA6FAD0EEB6FA4
:100F8000140EEC6F050EED6F140EEE6F630EEF6F27
:100F9000130EF06FC50EF16F120EF26F2D0EF36F80
:100FA000120EF46F990EF56F110EF66F0A0EF76FB1
:100FB000110EF86F800EF96F100EFA6FFA0EFB6FBC
:100FC0000F0EFC6F780EFD6F0F0EFE6FFA0EFF6FA7
:100FD0000E0E0101006F810E016F0E0E026F0B0EDF
:100FE000036F0E0E046F990E056F0D0E066F2B0E1C
:100FF000076F0D0E086FC00E096F0C0E0A6F580EAA
:101000000B6F0C0E0C6FF40E0D6F0B0E0E6F930E1C
:101010000F6F0B0E106F350E116F0B0E126FDA0E75
:10102000136F0A0E146F820E156F0A0E166F2C0EB8
:10103000176F0A0E186FDA0E196F090E1A6F8A0EE3
:101040001B6F090E1C6F3C0E1D6F090E1E6FF10EFB
:101050001F6F080E206FA90E216F080E226F620EFF
:10106000236F080E246F1E0E256F080E266FDC0EF0
:10107000276F070E286F9C0E296F070E2A6F5F0ED1
:101080002B6F070E2C6F230E2D6F070E2E6FE90EA0
:101090002F6F060E306FB10E316F060E326F7A0E63
:1010A000336F060E346F460E356F060E366F130E15
:1010B000376F060E386FE10E396F050E3A6FB20EBC
:1010C0003B6F050E3C6F830E3D6F050E3E6F570E56
:1010D0003F6F050E406F2B0E416F050E426F010EE4
:1010E000436F050E446FD90E456F040E466FB10E67
:1010F000476F040E486F8B0E496F040E4A6F660EE1
:101100004B6F040E4C6F430E4D6F040E4E6F200E4E
:101110004F6F040E506FFE0E516F030E526FDE0EB6
:10112000536F030E546FBF0E556F030E566FA00E14
:10113000576F030E586F830E596F030E5A6F660E6A
:101140005B6F030E5C6F4B0E5D6F030E5E6F300EB8
:101150005F6F030E606F160E616F030E626FFD0E00
:10116000636F020E646FE50E656F020E666FCD0E43
:10117000676F020E686FB60E696F020E6A6F00012C
:1011800012002A0E01016D6F6E6B020E146E0001CB
:10119000800E145C20E21404056E01EE6BF0D89012
:1011A0000534E926000EEA22EECF03F0EFCF04F07B
:1011B000050E0324016E000E0420026E01EE6BF09A
:1011C000D8901434E926000EEA2201C0EEFF02C0D6
:1011D000EFFF142ADCE1B80E02016D6F6E6BBA0EE0
:1011E0006F6F706BBB0E716F726BBC0E736F746B35
:1011F000BD0E756F766BBE0E776F786BBF0E796F15
:101200007A6BC10E7B6F7C6BC20E7D6F7E6BC30EE3
:101210007F6F806BC40E816F826BC50E836F846B92
:10122000C60E856F866BC80E876F886BC90E896F77
:101230008A6BCA0E8B6F8C6BCB0E8D6F8E6BCC0E48
:101240008F6F906BCD0E916F926BCF0E936F946BEF
:10125000D00E956F966BD10E976F986BD20E996FDB
:101260009A6BD30E9B6F9C6BD40E9D6F9E6BD60EAC
:101270009F6FA06BD70EA16FA26BD80EA36FA46B4C
:10128000D90EA56FA66BDA0EA76FA86BDB0EA96F40
:10129000AA6BDC0EAB6FAC6BDE0EAD6FAE6BDF0E10
:1012A000AF6FB06BE00EB16FB26BE10EB36FB46BAA
:1012B000E20EB56FB66BE30EB76FB86BE50EB96FA4
:1012C000BA6BE60EBB6FBC6BE70EBD6FBE6BE80E74
:1012D000BF6FC06BE90EC16FC26BEA0EC36FC46B08
:1012E000EC0EC56FC66BED0EC76FC86BEE0EC96F07
:1012F000CA6BEF0ECB6FCC6BF00ECD6FCE6BF10ED9
:10130000CF6FD06BF30ED16FD26BF40ED36FD46B63
:10131000F50ED56FD66BF60ED76FD86BF70ED96F6B
:10132000DA6BF80EDB6FDC6BF90EDD6FDE6BFB0E3C
:10133000DF6FE06BFC0EE16FE26BFD0EE36FE46BC1
:10134000FE0EE56FE66BE769E86BE96B010EEA6F8D
:10135000020EEB6F010EEC6F030EED6F010EEE6FE0
:10136000040EEF6F010EF06F050EF16F010EF26FBC
:10137000060EF36F010EF46F070EF56F010EF66F98
:10138000090EF76F010EF86F0A0EF96F010EFA6F72
:101390000B0EFB6F010EFC6F0C0EFD6F010EFE6F4E
:1013A0000D0EFF6F010E0301006F0E0E016F010E97
:1013B000026F100E036F010E046F110E056F010E08
:1013C000066F120E076F010E086F130E096F010EE4
:1013D0000A6F140E0B6F010E0C6F150E0D6F010EC0
:1013E0000E6F170E0F6F010E106F180E116F010E9A
:1013F000126F190E136F010E146F1A0E156F010E76
:10140000166F1B0E176F010E186F1C0E196F010E51
:101410001A6F1D0E1B6F010E1C6F1F0E1D6F010E2C
:101420001E6F200E1F6F010E206F210E216F010E07
:10143000226F220E236F010E246F230E256F010EE3
:10144000266F240E276F010E286F260E296F010EBE
:101450002A6F270E2B6F010E2C6F280E2D6F010E99
:101460002E6F290E2F6F010E306F2A0E316F010E75
:10147000326F2B0E336F010E346F2D0E356F010E50
:10148000366F2E0E376F010E386F2F0E396F010E2B
:101490003A6F300E3B6F010E3C6F310E3D6F010E07
:1014A0003E6F320E3F6F010E406F340E416F010EE2
:1014B000426F350E436F010E446F360E456F010EBD
:1014C000466F370E476F010E486F380E496F010E99
:1014D0004A6F390E4B6F010E4C6F3A0E4D6F010E75
:1014E0004E6F3C0E4F6F010E506F3D0E516F010E4F
:1014F000526F3E0E536F010E546F3F0E556F010E2B
:10150000566F400E576F010E586F410E596F010E06
:101510005A6F430E5B6F010E5C6F440E5D6F010EE0
:101520005E6F450E5F6F010E606F460E616F010EBC
:10153000626F470E636F010E646F480E656F010E98
:10154000666F4A0E676F010E686F4B0E696F010E72
:101550006A6F2F0E6D6F6E6B340E6F6F706B390E7E
:10156000716F726B3E0E736F746B420E756F766B9C
:10157000470E776F786B4C0E796F7A6B510E7B6FDD
:101580007C6B560E7D6F7E6B5B0E7F6F806B600E8B
:10159000816F826B650E836F846B690E856F866BBE
:1015A0006E0E876F886B730E896F8A6B780E8B6FE8
:1015B0008C6B7D0E8D6F8E6B820E8F6F906B870E96
:1015C000916F926B8C0E936F946B900E956F966BE0
:1015D000950E976F986B9A0E996F9A6B9F0E9B6FF3
:1015E0009C6BA40E9D6F9E6BA90E9F6FA06BAE0EA1
:1015F000A16FA26BB30EA36FA46BB70EA56FA66B02
:10160000BC0EA76FA86BC10EA96FAA6BC60EAB6FFD
:10161000AC6BCB0EAD6FAE6BD00EAF6FB06BD50EAB
:10162000B16FB26BDA0EB36FB46BDE0EB56FB66B23
:10163000E30EB76FB86BE80EB96FBA6BED0EBB6F08
:10164000BC6BF20EBD6FBE6BF70EBF6FC06BFC0EB6
:10165000C16FC26B010EC36FC46F050EC56F010E63
:10166000C66F0A0EC76F010EC86F0F0EC96F010E4D
:10167000CA6F140ECB6F010ECC6F190ECD6F010E19
:10168000CE6F1E0ECF6F010ED06F230ED16F010EE5
:10169000D26F280ED36F010ED46F2C0ED56F010EB2
:1016A000D66F310ED76F010ED86F360ED96F010E7F
:1016B000DA6F3B0EDB6F010EDC6F400EDD6F010E4B
:1016C000DE6F450EDF6F010EE06F4A0EE16F010E17
:1016D000E26F4F0EE36F010EE46F530EE56F010EE4
:1016E000E66F580EE76F010EE86F5D0EE96F010EB1
:1016F000EA6F620EEB6F010EEC6F670EED6F010E7D
:10170000EE6F6C0EEF6F010EF06F710EF16F010E48
:10171000F26F760EF36F010EF46F7A0EF56F010E15
:10172000F66F7F0EF76F010EF86F840EF96F010EE2
:10173000FA6F890EFB6F010EFC6F8E0EFD6F010EAE
:10174000FE6F930EFF6F010E0401006F980E016F84
:10175000010E026F9D0E036F010E046FA10E056F47
:10176000010E066FA60E076F010E086FAB0E096F14
:10177000010E0A6FB00E0B6F010E0C6FB50E0D6FE0
:10178000010E0E6FBA0E0F6F010E106FBF0E116FAC
:10179000010E126FC40E136F010E146FC80E156F79
:1017A000010E166FCD0E176F010E186FD20E196F46
:1017B000010E1A6FD70E1B6F010E1C6FDC0E1D6F12
:1017C000010E1E6FE10E1F6F010E206FE60E216FDE
:1017D000010E226FEB0E236F010E246FEF0E256FAB
:1017E000010E266FF40E276F010E286FF90E296F78
:1017F000010E2A6FFE0E2B6F010E2C6F030E2D6F44
:10180000020E2E6F080E2F6F020E306F0D0E316F0D
:10181000020E326F120E336F020E346F160E356FDA
:10182000020E366F1B0E376F020E386F200E396FA7
:10183000020E3A6F250E3B6F020E3C6F2A0E3D6F73
:10184000020E3E6F2F0E3F6F020E406F340E416F3F
:10185000020E426F390E436F020E446F3D0E456F0C
:10186000020E466F420E476F020E486F470E496FD9
:10187000020E4A6F4C0E4B6F020E4C6F510E4D6FA5
:10188000020E4E6F560E4F6F020E506F5B0E516F71
:10189000020E526F600E536F020E546F640E556F3E
:1018A000020E566F690E576F020E586F6E0E596F0B
:1018B000020E5A6F730E5B6F020E5C6F780E5D6FD7
:1018C000020E5E6F7D0E5F6F020E606F820E616FA3
:1018D000020E626F870E636F020E646F8B0E656F70
:1018E000020E666F900E676F020E686F950E696F3D
:1018F000020E6A6F2F0E6D6F6E6B340E6F6F706B12
:10190000390E716F726B3E0E736F746B420E756F92
:10191000766B470E776F786B4C0E796F7A6B510E42
:101920007B6F7C6B560E7D6F7E6B5B0E7F6F806B6B
:10193000600E816F826B650E836F846B690E856F9D
:10194000866B6E0E876F886B730E896F8A6B780E4D
:101950008B6F8C6B7D0E8D6F8E6B820E8F6F906B8D
:10196000870E916F926B8C0E936F946B900E956FA8
:10197000966B950E976F986B9A0E996F9A6B9F0E58
:101980009B6F9C6BA40E9D6F9E6BA90E9F6FA06BAF
:10199000AE0EA16FA26BB30EA36FA46BB70EA56FB3
:1019A000A66BBC0EA76FA86BC10EA96FAA6BC60E63
:1019B000AB6FAC6BCB0EAD6FAE6BD00EAF6FB06BD1
:1019C000D50EB16FB26BDA0EB36FB46BDE0EB56FBE
:1019D000B66BE30EB76FB86BE80EB96FBA6BED0E6E
:1019E000BB6FBC6BF20EBD6FBE6BF70EBF6FC06BF3
:1019F000FC0EC16FC26B010EC36FC46F050EC56FC5
:101A0000010EC66F0A0EC76F010EC86F0F0EC96FA9
:101A1000010ECA6F140ECB6F010ECC6F190ECD6F75
:101A2000010ECE6F1E0ECF6F010ED06F230ED16F41
:101A3000010ED26F280ED36F010ED46F2C0ED56F0E
:101A4000010ED66F310ED76F010ED86F360ED96FDB
:101A5000010EDA6F3B0EDB6F010EDC6F400EDD6FA7
:101A6000010EDE6F450EDF6F010EE06F4A0EE16F73
:101A7000010EE26F4F0EE36F010EE46F530EE56F40
:101A8000010EE66F580EE76F010EE86F5D0EE96F0D
:101A9000010EEA6F620EEB6F010EEC6F670EED6FD9
:101AA000010EEE6F6C0EEF6F010EF06F710EF16FA5
:101AB000010EF26F760EF36F010EF46F7A0EF56F72
:101AC000010EF66F7F0EF76F010EF86F840EF96F3F
:101AD000010EFA6F890EFB6F010EFC6F8E0EFD6F0B
:101AE000010EFE6F930EFF6F010E0501006F980E41
:101AF000016F010E026F9D0E036F010E046FA10EA8
:101B0000056F010E066FA60E076F010E086FAB0E74
:101B1000096F010E0A6FB00E0B6F010E0C6FB50E40
:101B20000D6F010E0E6FBA0E0F6F010E106FBF0E0C
:101B3000116F010E126FC40E136F010E146FC80ED9
:101B4000156F010E166FCD0E176F010E186FD20EA6
:101B5000196F010E1A6FD70E1B6F010E1C6FDC0E72
:101B60001D6F010E1E6FE10E1F6F010E206FE60E3E
:101B7000216F010E226FEB0E236F010E246FEF0E0B
:101B8000256F010E266FF40E276F010E286FF90ED8
:101B9000296F010E2A6FFE0E2B6F010E2C6F030EA4
:101BA0002D6F020E2E6F080E2F6F020E306F0D0E6E
:101BB000316F020E326F120E336F020E346F160E3B
:101BC000356F020E366F1B0E376F020E386F200E08
:101BD000396F020E3A6F250E3B6F020E3C6F2A0ED4
:101BE0003D6F020E3E6F2F0E3F6F020E406F340EA0
:101BF000416F020E426F390E436F020E446F3D0E6D
:101C0000456F020E466F420E476F020E486F470E39
:101C1000496F020E4A6F4C0E4B6F020E4C6F510E05
:101C20004D6F020E4E6F560E4F6F020E506F5B0ED1
:101C3000516F020E526F600E536F020E546F640E9E
:101C4000556F020E566F690E576F020E586F6E0E6B
:101C5000596F020E5A6F730E5B6F020E5C6F780E37
:101C60005D6F020E5E6F7D0E5F6F020E606F820E03
:101C7000616F020E626F870E636F020E646F8B0ED0
:101C8000656F020E666F900E676F020E686F950E9D
:101C9000696F020E6A6F510E6D6F6E6B530E6F6F30
:101CA000706B550E716F726B570E736F746B580EAD
:101CB000756F766B5A0E776F786B5C0E796F7A6BF7
:101CC0005E0E7B6F7C6B600E7D6F7E6B610E7F6F37
:101CD000806B630E816F826B650E836F846B670E02
:101CE000856F866B680E876F886B6A0E896F8A6B4B
:101CF0006C0E8B6F8C6B6E0E8D6F8E6B700E8F6F8C
:101D0000906B710E916F926B730E936F946B750E57
:101D1000956F966B770E976F986B780E996F9A6B9D
:101D20007A0E9B6F9C6B7C0E9D6F9E6B7E0E9F6FE1
:101D3000A06B800EA16FA26B810EA36FA46B830EAC
:101D4000A56FA66B850EA76FA86B870EA96FAA6BF0
:101D5000880EAB6FAC6B8A0EAD6FAE6B8C0EAF6F37
:101D6000B06B8E0EB16FB26B900EB36FB46B910E01
:101D7000B56FB66B930EB76FB86B950EB96FBA6B44
:101D8000970EBB6FBC6B980EBD6FBE6B9A0EBF6F8C
:101D9000C06B9C0EC16FC26B9E0EC36FC46BA00E56
:101DA000C56FC66BA10EC76FC86BA30EC96FCA6B98
:101DB000A50ECB6FCC6BA70ECD6FCE6BA90ECF6FE0
:101DC000D06BAA0ED16FD26BAC0ED36FD46BAE0EAC
:101DD000D56FD66BB00ED76FD86BB10ED96FDA6BEB
:101DE000B30EDB6FDC6BB50EDD6FDE6BB70EDF6F36
:101DF000E06BB90EE16FE26BBA0EE36FE46BBC0E01
:101E0000E56FE66BBE0EE76FE86BC00EE96FEA6B3D
:101E1000C10EEB6FEC6BC30EED6FEE6BC50EEF6F8B
:101E2000F06BC70EF16FF26BC90EF36FF46BCA0E55
:101E3000F56FF66BCC0EF76FF86BCE0EF96FFA6B91
:101E4000D00EFB6FFC6BD10EFD6FFE6BD30EFF6FE0
:101E50000601006BD50E016F026BD70E036F046B8A
:101E6000D90E056F066BDA0E076F086BDC0E096F73
:101E70000A6BDE0E0B6F0C6BE00E0D6F0E6BE10E3E
:101E80000F6F106BE30E116F126BE50E136F146B77
:101E9000E70E156F166BE90E176F186BEA0E196FC8
:101EA0001A6BEC0E1B6F1C6BEE0E1D6F1E6BF00E93
:101EB0001F6F206BF10E216F226BF30E236F246BCB
:101EC000F50E256F266BF70E276F286BF90E296F1D
:101ED0002A6BFA0E2B6F2C6BFC0E2D6F2E6BFE0EE9
:101EE0002F6F306B316B010E326F336F346F030E17
:101EF000356F010E366F050E376F010E386F070E06
:101F0000396F010E3A6F090E3B6F010E3C6F0A0EDE
:101F10003D6F010E3E6F0C0E3F6F010E406F0E0EB7
:101F2000416F010E426F100E436F010E446F120E8F
:101F3000456F010E466F130E476F010E486F150E69
:101F4000496F010E4A6F170E4B6F010E4C6F190E41
:101F50004D6F010E4E6F1A0E4F6F010E506F1C0E1B
:101F6000516F010E526F1E0E536F010E546F200EF3
:101F7000556F010E566F220E576F010E586F230ECC
:101F8000596F010E5A6F250E5B6F010E5C6F270EA5
:101F90005D6F010E5E6F290E5F6F010E606F2A0E7E
:101FA000616F010E626F2C0E636F010E646F2E0E57
:101FB000656F010E666F300E676F010E686F320E2F
:101FC000696F010E6A6F2F0E6D6F6E6B340E6F6F3F
:101FD000706B390E716F726B3E0E736F746B420EC5
:101FE000756F766B470E776F786B4C0E796F7A6BE7
:101FF000510E7B6F7C6B560E7D6F7E6B5B0E7F6F21
:10200000806B600E816F826B650E836F846B690ECF
:10201000856F866B6E0E876F886B730E896F8A6B08
:10202000780E8B6F8C6B7D0E8D6F8E6B820E8F6F2B
:10203000906B870E916F926B8C0E936F946B900EDA
:10204000956F966B950E976F986B9A0E996F9A6B2A
:102050009F0E9B6F9C6BA40E9D6F9E6BA90E9F6F36
:10206000A06BAE0EA16FA26BB30EA36FA46BB70EE5
:10207000A56FA66BBC0EA76FA86BC10EA96FAA6B4C
:10208000C60EAB6FAC6BCB0EAD6FAE6BD00EAF6F41
:10209000B06BD50EB16FB26BDA0EB36FB46BDE0EF0
:1020A000B56FB66BE30EB76FB86BE80EB96FBA6B6E
:1020B000ED0EBB6FBC6BF20EBD6FBE6BF70EBF6F4C
:1020C000C06BFC0EC16FC26B010EC36FC46F050EF7
:1020D000C56F010EC66F0A0EC76F010EC86F0F0ED7
:1020E000C96F010ECA6F140ECB6F010ECC6F190EA3
:1020F000CD6F010ECE6F1E0ECF6F010ED06F230E6F
:10210000D16F010ED26F280ED36F010ED46F2C0E3B
:10211000D56F010ED66F310ED76F010ED86F360E08
:10212000D96F010EDA6F3B0EDB6F010EDC6F400ED4
:10213000DD6F010EDE6F450EDF6F010EE06F4A0EA0
:10214000E16F010EE26F4F0EE36F010EE46F530E6D
:10215000E56F010EE66F580EE76F010EE86F5D0E3A
:10216000E96F010EEA6F620EEB6F010EEC6F670E06
:10217000ED6F010EEE6F6C0EEF6F010EF06F710ED2
:10218000F16F010EF26F760EF36F010EF46F7A0E9F
:10219000F56F010EF66F7F0EF76F010EF86F840E6C
:1021A000F96F010EFA6F890EFB6F010EFC6F8E0E38
:1021B000FD6F010EFE6F930EFF6F010E0701006FA2
:1021C000980E016F010E026F9D0E036F010E046FDA
:1021D000A10E056F010E066FA60E076F010E086FA8
:1021E000AB0E096F010E0A6FB00E0B6F010E0C6F74
:1021F000B50E0D6F010E0E6FBA0E0F6F010E106F40
:10220000BF0E116F010E126FC40E136F010E146F0B
:10221000C80E156F010E166FCD0E176F010E186FD9
:10222000D20E196F010E1A6FD70E1B6F010E1C6FA5
:10223000DC0E1D6F010E1E6FE10E1F6F010E206F71
:10224000E60E216F010E226FEB0E236F010E246F3D
:10225000EF0E256F010E266FF40E276F010E286F0B
:10226000F90E296F010E2A6FFE0E2B6F010E2C6FD7
:10227000030E2D6F020E2E6F080E2F6F020E306FA1
:102280000D0E316F020E326F120E336F020E346F6D
:10229000160E356F020E366F1B0E376F020E386F3B
:1022A000200E396F020E3A6F250E3B6F020E3C6F07
:1022B0002A0E3D6F020E3E6F2F0E3F6F020E406FD3
:1022C000340E416F020E426F390E436F020E446F9F
:1022D0003D0E456F020E466F420E476F020E486F6D
:1022E000470E496F020E4A6F4C0E4B6F020E4C6F39
:1022F000510E4D6F020E4E6F560E4F6F020E506F05
:102300005B0E516F020E526F600E536F020E546FD0
:10231000640E556F020E566F690E576F020E586F9E
:102320006E0E596F020E5A6F730E5B6F020E5C6F6A
:10233000780E5D6F020E5E6F7D0E5F6F020E606F36
:10234000820E616F020E626F870E636F020E646F02
:102350008B0E656F020E666F900E676F020E686FD0
:0E236000950E696F020E6A6F00011200FFD722
:020000040030CA
:0300010006170ED1
:020005008580F4
:060008000FC00FE00F40E5
:00000001FF
